:100000000C942A001895000018950000189500001F
:10001000189500001895000018950000189500002C
:10002000189500001895000018950000189500001C
:10003000189500000C940F241895000018950000E6
:1000400018950000189500001895000018950000FC
:10005000189500008FE58DBFC0E2E4E94E2E88E0E0
:100060008EBFD8E0F7E05F2EEEEFF7E0A0E6B0E05D
:10007000A89584B7082E877F84BF88E1992781BD22
:1000800091BD88278D933197E9F783E389B980E0A3
:1000900080BD88E18AB96624579AE0E0F0E0AFE9D4
:1000A000B0E00E940F2500919F00003011F00C94E9
:1000B0005C0084E180939F008A9A929A7894D29A05
:1000C000DA988C988D9A95988E9A96988F988A9AA5
:1000D0009298E1E0F0E0A6E8B2E00E940F25E2E0AD
:1000E000F0E0A1E9B2E00E940F25E3E0F0E0AAEF22
:1000F000B2E09CE00E941925D19AD998A19AA998BA
:10010000A69AAE9AD59AD69AD79AA7E0B3E0EAE92A
:10011000FAE40E942C230E94F32282E2A6E1B3E0DB
:100120008D9388278C930E94E0080E94EB080E9420
:1001300049090E9449095A924A9280E0A42DB52D9E
:100140008C9381E00E9489225A924A9280E0A42DE9
:10015000B52D8C9381E00E9489220E94DC092496AF
:1001600082E00E9485225A924A92A42DB52DE8EA97
:10017000FAE40E942C238CE00E9489220E948D0ABE
:1001800022968CE00E94852284E690E00E9417234C
:100190005A924A9280E0A42DB52D8C9381E00E9462
:1001A00089225A924A9281E0A42DB52D8C9381E048
:1001B0000E9489220E94DC09249682E00E94852206
:1001C0005A924A92E7E0F3E0A42DB52D0E94D9247B
:1001D0008FE00E9489220E948D0A22968FE00E9461
:1001E000852284E690E00E9417235A924A9280E08A
:1001F000A42DB52D8C9381E00E9489225A924A92B7
:1002000083E0A42DB52D8C9381E00E9489220E9469
:10021000DC09249682E00E9485225A924A92A42DFB
:10022000B52DE4EBFAE40E942C238FE00E94892292
:100230000E948D0A22968FE00E94852284E690E03B
:100240000E9417235A924A9280E0A42DB52D8C93D8
:1002500081E00E9489225A924A9284E0A42DB52D11
:100260008C9381E00E9489220E94DC09249682E01E
:100270000E9485225A924A92A42DB52DE4ECFAE40C
:100280000E942C238EE00E9489220E948D0A2296D1
:100290008EE00E9485225A924A9280E0A42DB52DCC
:1002A0008C9381E00E9489225A924A9285E0A42D83
:1002B000B52D8C9381E00E9489220E94DC0924964E
:1002C00082E00E9485225A924A92A42DB52DE4EB39
:1002D000FAE40E942C238FE00E9489220E948D0A5A
:1002E00022968FE00E948522E5E0F0E00E94E02265
:1002F000DA9A959A0E9449095A924A9280E0A42D6E
:10030000B52D8C9381E00E9489225A924A9282E014
:10031000A42DB52D8C9381E00E9489220E94DC09D6
:10032000249682E00E9485225A924A92A42DB52DED
:10033000E2EDFAE40E942C238FE00E9489220E94C1
:100340008D0A22968FE00E94852280E080938302AE
:100350005A924A9280E0A42DB52D8C9381E00E94A0
:1003600089225A924A9283E0A42DB52D8C9381E084
:100370000E9489220E94DC09249682E00E94852244
:100380005A924A92A42DB52DE2EEFAE40E942C2353
:100390008FE00E9489220E948D0A22968FE00E949F
:1003A00085228EE091E00E9417235A924A92809112
:1003B0008302A42DB52D8C9381E00E9489225A924C
:1003C0004A9283E0A42DB52D8C9381E00E9489226E
:1003D0000E94DC09249682E00E9485225A924A9269
:1003E000A42DB52DE2EFFAE40E942C2382E00E94B6
:1003F00089220E948D0A229682E00E9485228EE048
:1004000091E00E9417235A924A9280918302A42D70
:10041000B52D8C9381E00E9489225A924A9283E002
:10042000A42DB52D8C9381E00E9489220E94DC09C5
:10043000249682E00E9485225A924A92A42DB52DDC
:10044000E4EFFAE40E942C2382E00E9489220E94B9
:100450008D0A229682E00E9485228EE091E00E9421
:1004600017235A924A9280918302A42DB52D8C9322
:1004700081E00E9489225A924A9283E0A42DB52DF0
:100480008C9381E00E9489220E94DC09249682E0FC
:100490000E9485225A924A92A42DB52DE6EFFAE4E5
:1004A0000E942C2382E00E9489220E948D0A2296BB
:1004B00082E00E9485228EE091E00E9417235A92EA
:1004C0004A9280918302A42DB52D8C9381E00E94E5
:1004D00089225A924A9283E0A42DB52D8C9381E013
:1004E0000E9489220E94DC09249682E00E948522D3
:1004F0005A924A92A42DB52DE8EFFAE40E942C23DB
:1005000082E00E9489220E948D0A229682E00E9447
:1005100085228EE091E00E941723A3E8B2E08C913F
:100520008F5F8C9300918302023011F00C94D501FF
:100530009598DA985A924A9280E0A42DB52D8C9322
:1005400081E00E9489225A924A9282E0A42DB52D20
:100550008C9381E00E9489220E94DC09249682E02B
:100560000E9485225A924A92A42DB52DEAEFFAE410
:100570000E942C238FE00E9489220E948D0A2296DD
:100580008FE00E9485225A924A9280918302A42D84
:10059000B52D8C9381E00E9489225A924A9283E081
:1005A000A42DB52D8C9381E00E9489220E94DC0944
:1005B000249682E00E9485225A924A92A42DB52D5B
:1005C000EAE0FBE40E942C2382E00E9489220E9440
:1005D0008D0A229682E00E9485228EE091E00E94A0
:1005E00017235A924A9280918302A42DB52D8C93A1
:1005F00081E00E9489225A924A9283E0A42DB52D6F
:100600008C9381E00E9489220E94DC09249682E07A
:100610000E9485225A924A92A42DB52DE2EFFAE467
:100620000E942C2382E00E9489220E948D0A229639
:1006300082E00E9485228EE091E00E9417235A9268
:100640004A9280918302A42DB52D8C9381E00E9463
:1006500089225A924A9283E0A42DB52D8C9381E091
:100660000E9489220E94DC09249682E00E94852251
:100670005A924A92A42DB52DE4EFFAE40E942C235D
:1006800082E00E9489220E948D0A229682E00E94C6
:1006900085228EE091E00E9417235A924A9280911F
:1006A0008302A42DB52D8C9381E00E9489225A9259
:1006B0004A9283E0A42DB52D8C9381E00E9489227B
:1006C0000E94DC09249682E00E9485225A924A9276
:1006D000A42DB52DE6EFFAE40E942C2382E00E94BF
:1006E00089220E948D0A229682E00E9485228EE055
:1006F00091E00E9417235A924A9280918302A42D7E
:10070000B52D8C9381E00E9489225A924A9283E00F
:10071000A42DB52D8C9381E00E9489220E94DC09D2
:10072000249682E00E9485225A924A92A42DB52DE9
:10073000E8EFFAE40E942C2382E00E9489220E94C2
:100740008D0A229682E00E9485228EE091E00E942E
:100750001723A3E8B2E08C918F5F8C930091830202
:10076000063011F00C94C3025A924A9280E0A42DF4
:10077000B52D8C9381E00E9489225A924A9282E0A0
:10078000A42DB52D8C9381E00E9489220E94DC0962
:10079000249682E00E9485225A924A92A42DB52D79
:1007A000ECE0FBE40E942C238FE00E9489220E944F
:1007B0008D0A22968FE00E948522ECE1FBE40E94E4
:1007C000D2220E94D9225A924A9280918302A42D69
:1007D000B52D8C9381E00E9489225A924A9283E03F
:1007E000A42DB52D8C9381E00E9489220E94DC0902
:1007F000249682E00E9485225A924A92A42DB52D19
:10080000EAE0FBE40E942C2382E00E9489220E94FD
:100810008D0A229682E00E9485228EE091E00E945D
:100820001723ECE1FBE40E94D2220E94D9220E940D
:10083000F3155A924A9280918302A42DB52D8C9380
:1008400081E00E9489225A924A9283E0A42DB52D1C
:100850008C9381E00E9489220E94DC09249682E028
:100860000E9485225A924A92A42DB52DE2EFFAE415
:100870000E942C2382E00E9489220E948D0A2296E7
:1008800082E00E9485228EE091E00E9417235A9216
:100890004A9280918302A42DB52D8C9381E00E9411
:1008A00089225A924A9283E0A42DB52D8C9381E03F
:1008B0000E9489220E94DC09249682E00E948522FF
:1008C0005A924A92A42DB52DE4EFFAE40E942C230B
:1008D00082E00E9489220E948D0A229682E00E9474
:1008E00085228EE091E00E9417235A924A928091CD
:1008F0008302A42DB52D8C9381E00E9489225A9207
:100900004A9283E0A42DB52D8C9381E00E94892228
:100910000E94DC09249682E00E9485225A924A9223
:10092000A42DB52DE6EFFAE40E942C2382E00E946C
:1009300089220E948D0A229682E00E9485228EE002
:1009400091E00E9417235A924A9280918302A42D2B
:10095000B52D8C9381E00E9489225A924A9283E0BD
:10096000A42DB52D8C9381E00E9489220E94DC0980
:10097000249682E00E9485225A924A92A42DB52D97
:10098000E8EFFAE40E942C2382E00E9489220E9470
:100990008D0A229682E00E9485228EE091E00E94DC
:1009A0001723A3E8B2E08C918F5F8C935A924A92FE
:1009B00080E0A42DB52D8C9381E00E9489225A926B
:1009C0004A9282E0A42DB52D8C9381E00E94892269
:1009D0000E94DC09249682E00E9485225A924A9263
:1009E000A42DB52DE0E2FBE40E942C238FE00E94B1
:1009F00089220E948D0A22968FE00E9485225A92B7
:100A00004A9280918302A42DB52D8C9381E00E949F
:100A100089225A924A9283E0A42DB52D8C9381E0CD
:100A20000E9489220E94DC09249682E00E9485228D
:100A30005A924A92A42DB52DEAE0FBE40E942C23A1
:100A400082E00E9489220E948D0A229682E00E9402
:100A500085228EE091E00E9417235A924A9280915B
:100A60008302A42DB52D8C9381E00E9489225A9295
:100A70004A9283E0A42DB52D8C9381E00E948922B7
:100A80000E94DC09249682E00E9485225A924A92B2
:100A9000A42DB52DE2EFFAE40E942C2382E00E94FF
:100AA00089220E948D0A229682E00E9485228EE091
:100AB00091E00E941723ECE1FBE40E94D2220E9405
:100AC000D92288E290E00E941723AEE3B2E0BA9305
:100AD000AA930E94B5152296AEE3B2E0E0E3FBE4F0
:100AE0000E94392511F00C945B050E94F3155A926F
:100AF0004A9280918302A42DB52D8C9381E00E94AF
:100B000089225A924A9283E0A42DB52D8C9381E0DC
:100B10000E9489220E94DC09249682E00E9485229C
:100B20005A924A92A42DB52DE4EFFAE40E942C23A8
:100B300082E00E9489220E948D0A229682E00E9411
:100B400085228EE091E00E9417235A924A9280916A
:100B50008302A42DB52D8C9381E00E9489225A92A4
:100B60004A9283E0A42DB52D8C9381E00E948922C6
:100B70000E94DC09249682E00E9485225A924A92C1
:100B8000A42DB52DE6EFFAE40E942C2382E00E940A
:100B900089220E948D0A229682E00E9485228EE0A0
:100BA00091E00E9417235A924A9280918302A42DC9
:100BB000B52D8C9381E00E9489225A924A9283E05B
:100BC000A42DB52D8C9381E00E9489220E94DC091E
:100BD000249682E00E9485225A924A92A42DB52D35
:100BE000E8EFFAE40E942C2382E00E9489220E940E
:100BF0008D0A229682E00E9485228EE091E00E947A
:100C00001723A3E8B2E08C918F5F8C935A924A929B
:100C100080E0A42DB52D8C9381E00E9489225A9208
:100C20004A9282E0A42DB52D8C9381E00E94892206
:100C30000E94DC09249682E00E9485225A924A9200
:100C4000A42DB52DE4E3FBE40E942C238FE00E9449
:100C500089220E948D0A22968FE00E948522E4E478
:100C6000FBE40E94D22282E20E94DC22EEE4FBE45A
:100C70000E94D22282E20E94DC220E94D9225A9251
:100C80004A9280918302A42DB52D8C9381E00E941D
:100C900089225A924A9283E0A42DB52D8C9381E04B
:100CA0000E9489220E94DC09249682E00E9485220B
:100CB0005A924A92A42DB52DEAE0FBE40E942C231F
:100CC00082E00E9489220E948D0A229682E00E9480
:100CD00085228EE091E00E9417235A924A928091D9
:100CE0008302A42DB52D8C9381E00E9489225A9213
:100CF0004A9283E0A42DB52D8C9381E00E94892235
:100D00000E94DC09249682E00E9485225A924A922F
:100D1000A42DB52DE2EFFAE40E942C2382E00E947C
:100D200089220E948D0A229682E00E948522E2E0BA
:100D3000F0E00E94E0220E94F3158EE091E00E9414
:100D400017235A924A9280918302A42DB52D8C9339
:100D500081E00E9489225A924A9283E0A42DB52D07
:100D60008C9381E00E9489220E94DC09249682E013
:100D70000E9485225A924A92A42DB52DE4EFFAE4FE
:100D80000E942C2382E00E9489220E948D0A2296D2
:100D900082E00E9485228EE091E00E9417235A9201
:100DA0004A9280918302A42DB52D8C9381E00E94FC
:100DB00089225A924A9283E0A42DB52D8C9381E02A
:100DC0000E9489220E94DC09249682E00E948522EA
:100DD0005A924A92A42DB52DE6EFFAE40E942C23F4
:100DE00082E00E9489220E948D0A229682E00E945F
:100DF00085228EE091E00E9417235A924A928091B8
:100E00008302A42DB52D8C9381E00E9489225A92F1
:100E10004A9283E0A42DB52D8C9381E00E94892213
:100E20000E94DC09249682E00E9485225A924A920E
:100E3000A42DB52DE8EFFAE40E942C2382E00E9455
:100E400089220E948D0A229682E00E94852284E6F1
:100E500090E00E9417235A924A9280918302A42D17
:100E6000B52D8C9381E00E9489225A924A9283E0A8
:100E7000A42DB52D8C9381E00E9489220E94DC096B
:100E8000249682E00E948522A3E8B2E08C918F5FD5
:100E90008C935A924A9280918302A42DB52D8C9303
:100EA00081E00E9489225A924A9283E0A42DB52DB6
:100EB0008C9381E00E9489220E94DC09249682E0C2
:100EC0000E9485225A924A92A42DB52DEAE0FBE4B5
:100ED0000E942C2382E00E9489220E948D0A229681
:100EE00082E00E94852282E390E00E9417235A92BA
:100EF0004A9280918302A42DB52D8C9381E00E94AB
:100F000089225A924A9283E0A42DB52D8C9381E0D8
:100F10000E9489220E94DC09249682E00E94852298
:100F20005A924A92A42DB52DE2EFFAE40E942C23A6
:100F300082E00E9489220E948D0A229682E00E940D
:100F4000852282E390E00E9417235A924A92809170
:100F50008302A42DB52D8C9381E00E9489225A92A0
:100F60004A9283E0A42DB52D8C9381E00E948922C2
:100F70000E94DC09249682E00E9485225A924A92BD
:100F8000A42DB52DE4EFFAE40E942C2382E00E9408
:100F900089220E948D0A229682E00E94852282E3A5
:100FA00090E00E9417235A924A9280918302A42DC6
:100FB000B52D8C9381E00E9489225A924A9283E057
:100FC000A42DB52D8C9381E00E9489220E94DC091A
:100FD000249682E00E9485225A924A92A42DB52D31
:100FE000E6EFFAE40E942C2382E00E9489220E940C
:100FF0008D0A229682E00E94852282E390E00E9480
:1010000017235A924A9280918302A42DB52D8C9376
:1010100081E00E9489225A924A9283E0A42DB52D44
:101020008C9381E00E9489220E94DC09249682E050
:101030000E9485225A924A92A42DB52DE8EFFAE437
:101040000E942C2382E00E9489220E948D0A22960F
:1010500082E00E94852282E390E00E9417235A9248
:101060004A9280918302A42DB52D8C9381E00E9439
:1010700089225A924A9283E0A42DB52D8C9381E067
:101080000E9489220E94DC09249682E00E94852227
:101090005A924A92A42DB52DE6E5FBE40E942C233A
:1010A00082E00E9489220E948D0A229682E00E949C
:1010B000852282E390E00E941723A3E8B2E08C919E
:1010C0008F5F8C93009183020E3011F00C944907CE
:1010D00080E0809383020E9449095A924A9280E0FC
:1010E000A42DB52D8C9381E00E9489225A924A92B8
:1010F00082E0A42DB52D8C9381E00E9489220E946C
:10110000DC09249682E00E9485225A924A92A42DFC
:10111000B52DE8E5FBE40E942C238FE00E94892294
:101120000E948D0A22968FE00E9485220E94F3156C
:10113000DA9AE8E6FBE40E94D2220E94D92282E3F6
:1011400090E00E941723E2E7FBE40E94D2220E9473
:10115000D922E3E0F0E00E94E022DA980E94F31541
:1011600000919102013011F00C94C208ECE7FBE40D
:101170000E94D2220E94D92280E293E00E9417238B
:101180000E94F3150E944909DA9A0E94A1200E9448
:1011900003160E94FD210E9471170E94A91D0E9442
:1011A000291E0E94E81F0E94DE1A0E94E420DA989D
:1011B000EAE0F0E00E94E0220C94C408F894FFCF2B
:1011C000DF98EF93FF93E4EEF3E00E94E622FF91B5
:1011D000EF91DF9A0895DE98DD985A924A9281E263
:1011E000A42DB52D8C9381E00E9489220E94CA090A
:1011F000229681E00E9485225A924A9288ECA42D80
:10120000B52D8C9381E00E9489220E94CA09229602
:1012100081E00E9485225A924A9286E0A42DB52D43
:101220008C9381E00E9489220E94CA09229681E063
:101230000E9485225A924A9283E1A42DB52D8C9367
:1012400081E00E9489220E94CA09229681E00E94C0
:1012500085225A924A9280E2A42DB52D8C9381E08A
:101260000E9489220E94CA09229681E00E9485225A
:101270005A924A928CE0A42DB52D8C9381E00E9465
:1012800089220E94CA09229681E00E948522DE9A64
:10129000089582E00E942623DE98DD985A924A92B1
:1012A00080E2A42DB52D8C9381E00E9489220E94BA
:1012B000CA09229681E00E9485225A924A9280E8C9
:1012C000A42DB52D8C9381E00E9489220E94CA0929
:1012D000229681E00E9485225A924A9280E4A42DAF
:1012E000B52D8C9381E00E9489220E94CA09229622
:1012F00081E00E948522DD9A80E090E0A881B9819A
:101300008D939C93A881B9810D911C91073F51E069
:10131000150718F011F00C94A3095A924A9280E034
:10132000A42DB52D8C9381E00E9489220E94D309BF
:10133000229681E00E948522A881B9810E948D2297
:1013400010F40C948209DE9A82E0481A8827580A21
:10135000229608955A924A928DE0A42DB52D8C9331
:1013600081E00E9489220E94CA09229681E00E949F
:10137000852208955A924A928CE0A42DB52D8C9323
:1013800081E00E9489220E94CA09229681E00E947F
:1013900085220895DE98DD9891E0A881B9810E94A8
:1013A000E922DE9A0895DE98DD9A91E0A881B9815C
:1013B0000E94E922DE9A089581E00E9426235A9233
:1013C0004A9280E2A42DB52D8C9381E00E9489225F
:1013D0000E94CA09229681E00E948522EF93FF9322
:1013E000E4EEF3E00E94E622FF91EF91DE98DD98B3
:1013F000AC81BD810C9146E0049FA881B9810C921B
:10140000A881B9818C9180588C9391E0A881B98191
:101410000E94E922AA81BB810C9140E4040FA881BB
:10142000B9810C9391E0A881B9810E94E922DE9AEA
:1014300081E0481A8827580A2296089582E00E947F
:10144000262381E00E942623DE98DD985A924A9254
:1014500080E2A42DB52D8C9381E00E9489220E9408
:10146000CA09229681E00E9485225A924A9280E817
:10147000A42DB52D8C9381E00E9489220E94CA0977
:10148000229681E00E9485225A924A9280E4A42DFD
:10149000B52D8C9381E00E9489220E94CA09229670
:1014A00081E00E948522DD9A80E090E0AA81BB81E4
:1014B0008D939C93AA81BB810D911C91073F51E0B4
:1014C000150718F011F00C94860A0E948222A88158
:1014D000B9810E9432230C920E947F225A924A9232
:1014E000AA81BB818C91A42DB52D8C9381E00E94A3
:1014F00089220E94D309229681E00E948522AA8136
:10150000BB810E948D2210F40C945A0ADE9A83E06B
:10151000481A8827580A2496089581E00E942623B5
:1015200082E00E94262381E00E94262381E00E941F
:10153000262381E00E942623AA85BB850E943325AD
:10154000A885B9858C9381E0AC81BD818C93A885F9
:10155000B9854C91AC81BD810C91041718F011F044
:101560000C940E13AC81BD818C91EA85FB8501E062
:101570000A93AF81B8850E94DE24AE81BF81E4E882
:10158000FBE40E94392511F00C94CC0AEAE4F7E25E
:101590000E947F220C94C312E6E8FBE40E943925E6
:1015A00011F00C94D90AE0E5F7E20E947F220C9436
:1015B000C312E8E8FBE40E94392511F00C94E60A16
:1015C000E6E5F7E20E947F220C94C312EAE8FBE40E
:1015D0000E94392511F00C94F30AECE5F7E20E9421
:1015E0007F220C94C312ECE8FBE40E94392511F031
:1015F0000C94000BE2E6F7E20E947F220C94C312E7
:10160000EEE8FBE40E94392511F00C940D0BE8E69E
:10161000F7E20E947F220C94C312E0E9FBE40E94EF
:10162000392511F00C941A0BEEE6F7E20E947F22A6
:101630000C94C312E2E9FBE40E94392511F00C94EA
:10164000270BE4E7F7E20E947F220C94C312E4E93F
:10165000FBE40E94392511F00C94340BEAE7F7E221
:101660000E947F220C94C312E6E9FBE40E94392514
:1016700011F00C94410BE0E8F7E20E947F220C94F9
:10168000C312E8E9FBE40E94392511F00C944E0BDB
:10169000E6E8F7E20E947F220C94C312EAE9FBE439
:1016A0000E94392511F00C945B0BECE8F7E20E94E4
:1016B0007F220C94C312ECE9FBE40E94392511F05F
:1016C0000C94680BE2E9F7E20E947F220C94C312AB
:1016D000EEE9FBE40E94392511F00C94750BE8E962
:1016E000F7E20E947F220C94C312E0EAFBE40E941E
:1016F000392511F00C94820BEEE9F7E20E947F226B
:101700000C94C312E2EAFBE40E94392511F00C9418
:101710008F0BE4EAF7E20E947F220C94C312E4EA02
:10172000FBE40E94392511F00C949C0BEAEAF7E2E5
:101730000E947F220C94C312E6EAFBE40E94392542
:1017400011F00C94A90BE0EBF7E20E947F220C94BD
:10175000C312E8EAFBE40E94392511F00C94B60BA1
:10176000E6EBF7E20E947F220C94C312EAEAFBE464
:101770000E94392511F00C94C30BECEBF7E20E94A8
:101780007F220C94C312ECEAFBE40E94392511F08D
:101790000C94D00BE2ECF7E20E947F220C94C3126F
:1017A000EEEAFBE40E94392511F00C94DD0BE8EC25
:1017B000F7E20E947F220C94C312E0EBFBE40E944C
:1017C000392511F00C94EA0BEEECF7E20E947F222F
:1017D0000C94C312E2EBFBE40E94392511F00C9447
:1017E000F70BE4EDF7E20E947F220C94C312E4EBC6
:1017F000FBE40E94392511F00C94040CEAEDF7E2A9
:101800000E947F220C94C312E6EBFBE40E94392570
:1018100011F00C94110CE0EEF7E20E947F220C9480
:10182000C312E8EBFBE40E94392511F00C941E0C66
:10183000E6EEF7E20E947F220C94C312EAEBFBE48F
:101840000E94392511F00C942B0CECEEF7E20E946B
:101850007F220C94C312ECEBFBE40E94392511F0BB
:101860000C94380CE2EFF7E20E947F220C94C31232
:10187000EEEBFBE40E94392511F00C94450CE8EFE7
:10188000F7E20E947F220C94C312E0ECFBE40E947A
:10189000392511F00C94520CEEEFF7E20E947F22F2
:1018A0000C94C312E2ECFBE40E94392511F00C9475
:1018B0005F0CE4E0F8E20E947F220C94C312E4EC97
:1018C000FBE40E94392511F00C946C0CEAE0F8E27C
:1018D0000E947F220C94C312E6ECFBE40E9439259F
:1018E00011F00C94790CE0E1F8E20E947F220C9454
:1018F000C312E8ECFBE40E94392511F00C94860C2D
:10190000E6E1F8E20E947F220C94C312EAECFBE4C9
:101910000E94392511F00C94930CECE1F8E20E943E
:101920007F220C94C312ECECFBE40E94392511F0E9
:101930000C94A00CE2E2F8E20E947F220C94C31205
:10194000EEECFBE40E94392511F00C94AD0CE8E2BA
:10195000F8E20E947F220C94C312E0EDFBE40E94A7
:10196000392511F00C94BA0CEEE2F8E20E947F22C5
:101970000C94C312E2EDFBE40E94392511F00C94A3
:10198000C70CE4E3F8E20E947F220C94C312E4ED5A
:10199000FBE40E94392511F00C94D40CEAE3F8E240
:1019A0000E947F220C94C312E6EDFBE40E943925CD
:1019B00011F00C94E10CE0E4F8E20E947F220C9418
:1019C000C312E8EDFBE40E94392511F00C94EE0CF3
:1019D000E6E4F8E20E947F220C94C312EAEDFBE4F5
:1019E0000E94392511F00C94FB0CECE4F8E20E9403
:1019F0007F220C94C312ECEDFBE40E94392511F018
:101A00000C94080DE2E5F8E20E947F220C94C312C8
:101A1000EEEDFBE40E94392511F00C94150DE8E57C
:101A2000F8E20E947F220C94C312E0EEFBE40E94D5
:101A3000392511F00C94220DEEE5F8E20E947F2288
:101A40000C94C312E2EEFBE40E94392511F00C94D1
:101A50002F0DE4E6F8E20E947F220C94C312E4EE1C
:101A6000FBE40E94392511F00C943C0DEAE6F8E203
:101A70000E947F220C94C312E6EEFBE40E943925FB
:101A800011F00C94490DE0E7F8E20E947F220C94DB
:101A9000C312E8EEFBE40E94392511F00C94560DB8
:101AA000E6E7F8E20E947F220C94C312EAEEFBE420
:101AB0000E94392511F00C94630DECE7F8E20E94C6
:101AC0007F220C94C312ECEEFBE40E94392511F046
:101AD0000C94700DE2E8F8E20E947F220C94C3128D
:101AE000EEEEFBE40E94392511F00C947D0DE8E840
:101AF000F8E20E947F220C94C312E0EFFBE40E9404
:101B0000392511F00C948A0DEEE8F8E20E947F224C
:101B10000C94C312E2EFFBE40E94392511F00C94FF
:101B2000970DE4E9F8E20E947F220C94C312E4EFDF
:101B3000FBE40E94392511F00C94A40DEAE9F8E2C7
:101B40000E947F220C94C312E6EFFBE40E94392529
:101B500011F00C94B10DE0EAF8E20E947F220C949F
:101B6000C312E8EFFBE40E94392511F00C94BE0D7E
:101B7000E6EAF8E20E947F220C94C312EAEFFBE44B
:101B80000E94392511F00C94CB0DECEAF8E20E948A
:101B90007F220C94C312ECEFFBE40E94392511F074
:101BA0000C94D80DE2EBF8E20E947F220C94C31251
:101BB000EEEFFBE40E94392511F00C94E50DE8EB03
:101BC000F8E20E947F220C94C312E0E0FCE40E9441
:101BD000392511F00C94F20DE6E8F7E20E947F221D
:101BE0000C94C312E2E0FCE40E94392511F00C943D
:101BF000FF0DE2E2F8E20E947F220C94C312E4E0BF
:101C0000FCE40E94392511F00C940C0EEAE2F6E295
:101C10000E947F220C94C312E6E0FCE40E94392566
:101C200011F00C94190EE0E3F6E20E947F220C946E
:101C3000C312E8E0FCE40E94392511F00C94260E52
:101C4000E6E3F6E20E947F220C94C312EAE0FCE491
:101C50000E94392511F00C94330EECE3F6E20E9459
:101C60007F220C94C312ECE0FCE40E94392511F0B1
:101C70000C94400EE2E4F6E20E947F220C94C31220
:101C8000EEE0FCE40E94392511F00C944D0EE8E4DE
:101C9000F6E20E947F220C94C312E0E1FCE40E9471
:101CA000392511F00C945A0EEEE4F6E20E947F22E0
:101CB0000C94C312E2E1FCE40E94392511F00C946B
:101CC000670EE4E5F6E20E947F220C94C312E4E181
:101CD000FCE40E94392511F00C94740EEEE9F7E251
:101CE0000E947F220C94C312E6E1FCE40E94392595
:101CF00011F00C94810EEAE3F8E20E947F220C942A
:101D0000C312E8E1FCE40E94392511F00C948E0E18
:101D1000EAE5F6E20E947F220C94C312EAE1FCE4B9
:101D20000E94392511F00C949B0EE0E6F6E20E9429
:101D30007F220C94C312ECE1FCE40E94392511F0DF
:101D40000C94A80EE6E6F6E20E947F220C94C312E1
:101D5000EEE1FCE40E94392511F00C94B50EECE69E
:101D6000F6E20E947F220C94C312E0E2FCE40E949F
:101D7000392511F00C94C20EE2E7F6E20E947F22B0
:101D80000C94C312E2E2FCE40E94392511F00C9499
:101D9000CF0EE8E7F6E20E947F220C94C312E4E241
:101DA000FCE40E94392511F00C94DC0EEEE7F6E21B
:101DB0000E947F220C94C312E6E2FCE40E943925C3
:101DC00011F00C94E90EE4E8F6E20E947F220C94F4
:101DD000C312E6E5FBE40E94392511F00C94F60EDF
:101DE000EAE8F6E20E947F220C94C312E8E2FCE4E7
:101DF0000E94392511F00C94030FE0E9F6E20E94ED
:101E00007F220C94C312EAE2FCE40E94392511F00F
:101E10000C94100FE2ECF7E20E947F220C94C312A4
:101E2000ECE2FCE40E94392511F00C941D0FE6E968
:101E3000F6E20E947F220C94C312EEE2FCE40E94C0
:101E4000392511F00C942A0FECE9F6E20E947F226A
:101E50000C94C312E0E3FCE40E94392511F00C94C9
:101E6000370FE2EAF6E20E947F220C94C312E2E30B
:101E7000FCE40E94392511F00C94440FEEECF7E2DB
:101E80000E947F220C94C312E4E3FCE40E943925F3
:101E900011F00C94510FE8EAF6E20E947F220C94B4
:101EA000C312E6E3FCE40E94392511F00C945E0FA6
:101EB000E0EBF7E20E947F220C94C312E8E3FCE41B
:101EC0000E94392511F00C946B0FEEEAF6E20E94A5
:101ED0007F220C94C312EAE3FCE40E94392511F03E
:101EE0000C94780FEAEDF7E20E947F220C94C31263
:101EF000ECE3FCE40E94392511F00C94850FE6E731
:101F0000F8E20E947F220C94C312EEE3FCE40E94EC
:101F1000392511F00C94920FE4EBF6E20E947F2237
:101F20000C94C312E0E4FCE40E94392511F00C94F7
:101F30009F0FEAEBF6E20E947F220C94C312E2E4C8
:101F4000FCE40E94392511F00C94AC0FE0EEF7E2AE
:101F50000E947F220C94C312E4E4FCE40E94392521
:101F600011F00C94B90FECE7F8E20E947F220C9478
:101F7000C312E6E4FCE40E94392511F00C94C60F6C
:101F8000E2E9F7E20E947F220C94C312E8E4FCE449
:101F90000E94392511F00C94D30FEEE2F8E20E9472
:101FA0007F220C94C312EAE4FCE40E94392511F06C
:101FB0000C94E00FE8EFF7E20E947F220C94C3122A
:101FC000ECE4FCE40E94392511F00C94ED0FE0ECF8
:101FD000F6E20E947F220C94C312EEE4FCE40E941D
:101FE000392511F00C94FA0FE6ECF6E20E947F22FC
:101FF0000C94C312E0E5FCE40E94392511F00C9426
:102000000710E2EBF8E20E947F220C94C312E2E593
:10201000FCE40E94392511F00C941410E0E1F8E280
:102020000E947F220C94C312E4E5FCE40E9439254F
:1020300011F00C942110ECEAF8E20E947F220C943B
:10204000C312E8EFFAE40E94392511F00C942E1027
:10205000ECECF6E20E947F220C94C312E6E5FCE46D
:102060000E94392511F00C943B10E2EDF6E20E943B
:102070007F220C94C312E6EFFAE40E94392511F096
:102080000C944810E4EEF6E20E947F220C94C312F6
:10209000E8E5FCE40E94392511F00C945510EAEEB5
:1020A000F6E20E947F220C94C312EAE5FCE40E944F
:1020B000392511F00C946210E8EDF6E20E947F22BF
:1020C0000C94C312ECE5FCE40E94392511F00C9449
:1020D0006F10EEEDF6E20E947F220C94C312E4EF43
:1020E000FAE40E94392511F00C947C10E0EFF6E23E
:1020F0000E947F220C94C312EEE5FCE40E94392575
:1021000011F00C948910E6EFF6E20E947F220C9405
:10211000C312E2EFFAE40E94392511F00C949610F4
:10212000ECEFF6E20E947F220C94C312E0E6FCE49E
:102130000E94392511F00C94A310E2E0F7E20E940E
:102140007F220C94C312E2E6FCE40E94392511F0D0
:102150000C94B010E8E2F8E20E947F220C94C312C3
:10216000E4E6FCE40E94392511F00C94BD10E8E08F
:10217000F7E20E947F220C94C312EAE0FBE40E9483
:10218000392511F00C94CA10EEE0F7E20E947F228C
:102190000C94C312E6E6FCE40E94392511F00C947D
:1021A000D710E4E1F7E20E947F220C94C312E8E624
:1021B000FCE40E94392511F00C94E410EAE1F7E206
:1021C0000E947F220C94C312EAE6FCE40E943925A7
:1021D00011F00C94F110E0E2F7E20E947F220C94DF
:1021E000C312ECE6FCE40E94392511F00C94FE10B9
:1021F000E6E2F7E20E947F220C94C312EEE6FCE4D2
:102200000E94392511F00C940B11ECE2F7E20E94C8
:102210007F220C94C312E0E7FCE40E94392511F000
:102220000C941811E2E3F7E20E947F220C94C3128F
:10223000E2E7FCE40E94392511F00C942511E8E353
:10224000F7E20E947F220C94C312E4E7FCE40E94B0
:10225000392511F00C943211EEE3F7E20E947F224F
:102260000C94C312E6E7FCE40E94392511F00C94AB
:102270003F11E4E4F7E20E947F220C94C312E8E7E6
:10228000FCE40E94392511F00C944C11EEEBF8E2BD
:102290000E947F220C94C312EAE7FCE40E943925D5
:1022A00011F00C945911EAECF8E20E947F220C9490
:1022B000C312ECE7FCE40E94392511F00C9466117E
:1022C000E4ECF8E20E947F220C94C312EEE7FCE4F7
:1022D0000E94392511F00C947311E0EDF8E20E9490
:1022E0007F220C94C312E0E8FCE40E94392511F02F
:1022F0000C948011E6E0F9E20E947F220C94C31254
:10230000E2E8FCE40E94392511F00C948D11E6ED11
:10231000F8E20E947F220C94C312E4E8FCE40E94DD
:10232000392511F00C949A11E8E1F9E20E947F221C
:102330000C94C312E6E8FCE40E94392511F00C94D9
:10234000A711ECE3F9E20E947F220C94C312E8E8A3
:10235000FCE40E94392511F00C94B411E2E4F9E296
:102360000E947F220C94C312EAE8FCE40E94392503
:1023700011F00C94C111E0E0F9E20E947F220C946C
:10238000C312ECE8FCE40E94392511F00C94CE1144
:10239000E4E5F9E20E947F220C94C312EEE8FCE42B
:1023A0000E94392511F00C94DB11E0E6F9E20E945D
:1023B0007F220C94C312E0E9FCE40E94392511F05D
:1023C0000C94E811E0E3F9E20E947F220C94C3121E
:1023D000E2E9FCE40E94392511F00C94F511ECE0DF
:1023E000F9E20E947F220C94C312E4E9FCE40E940B
:1023F000392511F00C940212EEE1F9E20E947F22DD
:102400000C94C312E6E9FCE40E94392511F00C9407
:102410000F12E8EEF8E20E947F220C94C312E8E962
:10242000FCE40E94392511F00C941C12EAE2F9E256
:102430000E947F220C94C312EAE9FCE40E94392531
:1024400011F00C942912E8E4F9E20E947F220C9426
:10245000C312ECE9FCE40E94392511F00C94361209
:10246000ECEDF8E20E947F220C94C312EEE9FCE44A
:102470000E94392511F00C944312E6E3F9E20E9420
:102480007F220C94C312E0EAFCE40E94392511F08B
:102490000C945012EAE5F9E20E947F220C94C312D8
:1024A000E2EAFCE40E94392511F00C945D12EEEE94
:1024B000F8E20E947F220C94C312E4EAFCE40E943A
:1024C000392511F00C946A12E2E1F9E20E947F22B0
:1024D0000C94C312E6E1F3E00E943B2511F00C944A
:1024E0007712E4E2F9E20E947F220C94C312E6EA3A
:1024F000FCE40E94392511F00C948412EEE4F9E218
:102500000E947F220C94C312E8EAFCE40E94392561
:1025100011F00C949112E2EEF8E20E947F220C94EA
:10252000C312EAEAFCE40E94392511F00C949E12D1
:10253000EAEFF8E20E947F220C94C312ECEAFCE47A
:102540000E94392511F00C94AB12E6E6F9E20E94E4
:102550007F220C94C312EEEAFCE40E94392511F0AC
:102560000C94B812ECE6F9E20E947F220C94C3129C
:10257000E0EBFCE40E94392511F00C94C312E4EF67
:10258000F8E20E947F2281E0AA81BB818C93AA811C
:10259000BB810C91053018F011F00C94F1120E94DF
:1025A0008222A881B9810E9432230C920E947F224C
:1025B0005A924A92AA81BB818C91A42DB52D8C93FD
:1025C00081E00E9489220E94D309229681E00E9424
:1025D0008522AA81BB818C918F5F8C9310F40C941F
:1025E000C71280E0A881B9818C935A924A92AA813D
:1025F000BB818C91A42DB52D8C9381E00E94892202
:102600000E94D309229681E00E948522AC81BD817F
:102610008C918F5F8C9310F40C94A70ADE9A86E05D
:10262000481A8827580A2A9608957F49494931004F
:102630007C4A4A4931007F49494936007C54542834
:1026400000007F01010103007C0404040C00E05140
:102650004F41FF00E0544C44FC007C55545544006D
:1026600038555455180077087F0877006C107C1097
:102670006C004149494936004454545428007F10A5
:1026800008047F007C2010087C007F7F7F7F7F0014
:102690007842241278007C102844000020413F0139
:1026A0007F0020443C047C007C0810087C007C10E7
:1026B00010107C007F0101017F007C0404047C0079
:1026C00004047C0404004728100807007F7F7F7FF4
:1026D0007F000C1010107C000C127F120C001824CC
:1026E0007E2418007F7F7F7F41007C404040FC00BB
:1026F0007F7F7F4141007C4078407C007F7F41416B
:1027000041007C407840FC007C50502000007F411C
:1027100041414100414141414100414141417F002E
:102720007C5020007C00224149493E0028445454FA
:1027300038007F083E413E007C103844380046296E
:1027400019097F00085434147C003E5149453E006D
:1027500000427F4000004261514946002241494900
:1027600036001814127F10002745454539003E49B0
:1027700049493200611109050300364949493600CB
:10278000264949493E007E0909097E007F49494999
:1027900036003E41414122007F4141413E007F4998
:1027A000494941007F09090901003E4149493A0070
:1027B0007F0808087F0000417F410000204141411F
:1027C0003F007F08142241007F40404040007F02CC
:1027D00004027F007F0408107F003E4141413E001B
:1027E0007F09090906003E4151617E007F091929D0
:1027F000460006494949300001017F0101003F4080
:1028000040403F001F2040201F007F2010207F00FD
:1028100063140814630003047804030061514945FC
:1028200043002054545478007F48444438003844CE
:1028300044442800384444487F0038545454180015
:1028400000047E0500000C52524A3C007F0804043C
:10285000780000447D4000000040443D00007F209F
:102860001028440000417F4000007C0418047C00D4
:102870007C08040478003844444438007C14242440
:102880001800182424147C007C0404080000085458
:1028900054542000043F444000003C4040407C0031
:1028A0001C2040201C003C4030403C0044281028A4
:1028B00044000C5050483C004464544C4400000018
:1028C0000000000000606000000008080808080020
:1028D000003636000000000609090600007F41416D
:1028E00000000041417F0000552A552A5500070984
:1028F0007F0907004040404040000056360000007D
:102900004040007070004040000000001414141497
:1029100014000201510906007C7C00000000000048
:102920005F000000000700070000147F147F140000
:102930002214081422002313086462007C7C007FA8
:102940007F00000503000000001C22410000004140
:10295000221C000014083E08140008083E08080065
:10296000000050300000201008040200020408108B
:102970002000000000000000000000000000000037
:102980000080E0F8F8F8F0C0000008081838F8F8FF
:10299000F8F8F808080000000000000808F8F878C7
:1029A000180808000808D8F8F8F8F878080808089F
:1029B00018F8F8F0F0E0000000008888888888881F
:1029C0008888F800000000000000000000000000FF
:1029D0000000C0F03E0F01030F3FFFFFFEF8E000D4
:1029E000000001071FFFFFFFFCF080000000C0F89F
:1029F0001F0701000000000080F8FFFFFF7F276035
:102A0000E0E0F0F8DC1F0F0F070100000000784441
:102A10004444447850484400000000000000000096
:102A20008080C0E0F8FEC78181010101010181873A
:102A3000FFFFFFFFFCE0C0808000031F7FFFFFFE61
:102A40007C0F0300000000808080C0F8FFFFFFFFC4
:102A5000CF80800001071F7FFFFFFCF0C080800057
:102A600000007C040808102020407D0000000000C9
:102A7000000000000000000000000808F8F8F80856
:102A80000000000000000000000000000000000046
:102A900000000000001818180000000000000000EE
:102AA0000000000000000000000000000000000026
:102AB0000000000000003E222222222222223E00AC
:102AC0000000000000000000F8FCFE070181F1FF9B
:102AD000FF1F000078FCFE9311190F8F46808E9E19
:102AE0001F39F9F3E30301E1FFFF1F000000F8FCC9
:102AF000FE070301E1FEFF1F010181FFFF7F0602C8
:102B0000F1FFFF1E0000000000009F909090909049
:102B100090909F00000000000000000000010101F3
:102B2000010000010101010000000101010101009B
:102B3000000001010101010000000000010101018C
:102B400000000C1D1911191F0F07010000000101E1
:102B50000100000000010101010000000000101050
:102B60001010101010101F000000A881B9818827D4
:102B70008C930E94A122ADE0B1E08C9300910D01F5
:102B8000003011F00C94C6150C94F0150D3011F0B6
:102B90000C94CC150C94F0150A3011F00C94DB1544
:102BA000A881B9818C91803011F40C94D9150C94C2
:102BB000F2150C94F01500910D010F3118F011F081
:102BC0000C94E4150C94F015ADE0B1E08C91A88163
:102BD000B9818F930E9494228F918D9388278C9333
:102BE0000C94B915089584E690E00E9417230E9482
:102BF000A122ADE0B1E08C9300910D01003011F005
:102C00000C94F71508950E949B22AEE0B1E08C93DE
:102C100000910E01013011F00C947017AEE3B2E098
:102C2000BA93AA930E94B5152296EEE3F2E004E06F
:102C3000AFE0B1E00E94E524AFE0B1E0E2EBFCE4FC
:102C40000E94392511F00C946A17AEE3B2E00E949D
:102C50003325EA2FFB2F3397F0400FEFAFE1B1E0C0
:102C60000E94E524EFE1F1E001E0A2E2B1E00E9480
:102C7000E524A2E2B1E0EEE8FCE40E94392511F07F
:102C80000C944F16AEE3B2E00E943325EA2FFB2FDF
:102C90003297F0400FEFAFE1B1E00E94E524E1E0B0
:102CA000F0E00E94E022ABEAB0E088278C93E8EBEA
:102CB000FCE40E94D222AFE1B1E00E94CC220E944B
:102CC000D9228AE090E00E941723AEE3B2E0BA93E3
:102CD000AA930E94B51522968AE090E00E941723DD
:102CE000AEE3B2E0BA93AA930E94B515229686E1AC
:102CF000EEE3F2E00CE00A93ABEAB0E00E94DE24DF
:102D0000EEE3F2E0A4E2B1E00E94D9248AE090E090
:102D10000E941723AEE3B2E0BA93AA930E94B515BE
:102D20002296EEE3F2E0A4E2B1E00E94D924E4E2CC
:102D3000F1E00EE0A4E2B1E00E94E524DA9884E636
:102D400090E00E941723DA9A82E390E00E94172312
:102D5000A3E8B2E08C918F5F8C93009183020A30DC
:102D600011F00C949E1680E0809383025A924A924E
:102D700080E0A42DB52D8C9381E00E9489225A9287
:102D80004A9282E0A42DB52D8C9381E00E94892285
:102D90000E94DC09249682E00E9485225A924A927F
:102DA000A42DB52DE2ECFCE40E942C238FE00E94C0
:102DB00089220E948D0A22968FE00E9485225A92D3
:102DC0004A9280E0A42DB52D8C9381E00E94892247
:102DD0005A924A9282E0A42DB52D8C9381E00E94F4
:102DE00089220E94DC09249682E00E9485225A9260
:102DF0004A92EBEAF0E0A42DB52D0E94D9248CE094
:102E00000E9489220E948D0A22968CE00E948522CF
:102E10005A924A9280E0A42DB52D8C9381E00E94B5
:102E200089225A924A9283E0A42DB52D8C9381E099
:102E30000E9489220E94DC09249682E00E94852259
:102E40005A924A92A42DB52DE2ECFCE40E942C2368
:102E50008FE00E9489220E948D0A22968FE00E94B4
:102E600085225A924A9280E0A42DB52D8C9381E060
:102E70000E9489225A924A9283E0A42DB52D8C9308
:102E800081E00E9489220E94DC09249682E00E944F
:102E900085225A924A92E4E2F1E0A42DB52D0E94D7
:102EA000D92489E70E9489220E948D0A229689E707
:102EB0000E948522E4E4FBE40E94D22282E20E9486
:102EC000DC22EEE4FBE40E94D22282E20E94DC22B9
:102ED0000E94D92284E690E00E9417230E94F315F5
:102EE0000895A4E2B1E0E4E8FBE40E94392511F082
:102EF0000C94DD17969892988091AA008F7B80930E
:102F0000AA00A7E8B2E0E2EDFCE40E942C23A4E2D0
:102F1000B1E088278C935A924A9280E0A42DB52D77
:102F20008C9381E00E9489225A924A9282E0A42DD9
:102F3000B52D8C9381E00E9489220E94DC092496A1
:102F400082E00E9485225A924A92A42DB52DE6ED88
:102F5000FCE40E942C238FE00E9489220E948D0AAB
:102F600022968FE00E9485225A924A9280E0A42DF8
:102F7000B52D8C9381E00E9489225A924A9283E077
:102F8000A42DB52D8C9381E00E9489220E94DC093A
:102F9000249682E00E9485225A924A92A42DB52D51
:102FA000E6EEFCE40E942C238FE00E9489220E941E
:102FB0008D0A22968FE00E948522A4E2B1E0E6E825
:102FC000FBE40E94392511F00C94E118969A5A926C
:102FD0004A9280E0A42DB52D8C9381E00E94892235
:102FE0005A924A9283E0A42DB52D8C9381E00E94E1
:102FF00089220E94DC09249682E00E9485225A924E
:103000004A92A42DB52DE6EFFCE40E942C238FE01C
:103010000E9489220E948D0A22968FE00E948522BA
:1030200088E28093EA02ABEEB2E0EAEEF2E00E94C0
:103030005D2480E10E942623EBEEF2E0A881B981B5
:103040000E94D924ABEEB2E0E6E0FDE40E942C231E
:10305000ABEEB2E00E949422E8E7FCE40E942C234D
:10306000E881F981ABEEB2E00E9494220E94D9245B
:10307000ABEEB2E00E949422E0EDFBE40E942C2330
:1030800080E1481A8827580A22965A924A9280E08C
:10309000A42DB52D8C9381E00E9489225A924A92E8
:1030A00082E0A42DB52D8C9381E00E9489220E949C
:1030B000DC09249682E00E9485225A924A92A42D2D
:1030C000B52DE2ECFCE40E942C238FE00E948922C3
:1030D0000E948D0A22968FE00E9485225A924A927F
:1030E00080E0A42DB52D8C9381E00E9489225A9214
:1030F0004A9282E0A42DB52D8C9381E00E94892212
:103100000E94DC09249682E00E9485225A924A920B
:10311000EBEEF2E0A42DB52D0E94D9248FE00E94A1
:1031200089220E948D0A22968FE00E948522E1E08A
:10313000F0E00E94E0228091EA0281508093EA024E
:103140000091EA02003011F00C941318929A8091C9
:10315000AA0080648093AA00A7E8B2E0E2E1FDE45F
:103160000E942C23A4E2B1E088278C935A924A92C1
:1031700080E0A42DB52D8C9381E00E9489225A9283
:103180004A9282E0A42DB52D8C9381E00E94892281
:103190000E94DC09249682E00E9485225A924A927B
:1031A000A42DB52DE6E1FDE40E942C238FE00E94C2
:1031B00089220E948D0A22968FE00E9485220E9419
:1031C000F315A4E2B1E0E8E8FBE40E94392511F030
:1031D0000C94F4180E946220A4E2B1E088278C933A
:1031E000ABEAB0E088278C93A4E2B1E0EAE8FBE424
:1031F0000E94392511F00C9407190E947720A4E24F
:10320000B1E088278C93ABEAB0E088278C93A4E2E6
:10321000B1E0ECE8FBE40E94392511F00C9424198C
:103220000E94DE1AE3E9F2E0ADE9B1E00E94D924A0
:10323000EDE9F2E0ADE9B1E00E9494220E94D924C8
:103240000E949C1A0E94F315A4E2B1E0EEE8FBE4B0
:103250000E94392511F00C943B1980E0809386027E
:10326000E1E0F0E0A6E8B2E07BE70E94F324A4E20C
:10327000B1E088278C93A4E2B1E0E0E9FBE40E948E
:10328000392511F00C94521981E080938602E1E017
:10329000F0E0A6E8B2E07BE70E94F324A4E2B1E00C
:1032A00088278C93A4E2B1E0E2E9FBE40E9439258F
:1032B00011F00C946519E6E2FDE40E94D2220E940E
:1032C000D922A4E2B1E088278C93A4E2B1E0E4E93A
:1032D000FBE40E94392511F00C947819ECE7FBE42B
:1032E0000E94D2220E94D922A4E2B1E088278C93C6
:1032F000A4E2B1E0EEE2FDE40E94392511F00C9465
:10330000AA19EBEAF0E0AAEFB2E00E94D924E3E0C8
:10331000F0E0AAEFB2E07BE70E940425ADE9B1E05E
:10332000EAE3FDE40E942C23EAEFF2E0ADE9B1E02C
:103330000E9494220E94D924ADE9B1E00E94942217
:10334000E4E4FDE40E942C230E949C1AA4E2B1E074
:1033500088278C93A4E2B1E0E4EAFCE40E943925DA
:1033600011F00C944F1AA6EAB0E0EFE9F0E00E94E9
:103370005D24ADE9B1E0E8E4FDE40E942C238AE09D
:10338000ADE9B1E08F930E9494228F918D938827AD
:103390008C93ADE9B1E00E949422E0E5FDE40E9447
:1033A0002C23E3E9F2E0ADE9B1E00E9494220E940F
:1033B000D924EDE9F2E0ADE9B1E00E9494220E9447
:1033C000D9248AE0ADE9B1E08F930E9494228F91D5
:1033D0008D9388278C93ADE9B1E00E949422E6E5B5
:1033E000FDE40E942C23E6EAF0E0ADE9B1E00E94A2
:1033F00094220E94D9248AE0ADE9B1E08F930E9423
:1034000094228F918D9388278C93ADE9B1E00E942F
:103410009422ECE5FDE40E942C23E7E8F2E0ADE91C
:10342000B1E00E9494220E94D9248AE0ADE9B1E083
:103430008F930E9494228F918D9388278C93ADE96E
:10344000B1E00E949422E2E6FDE40E942C23EBE826
:10345000F2E0ADE9B1E00E9494220E94D9248AE012
:10346000ADE9B1E08F930E9494228F918D938827CC
:103470008C93ADE9B1E00E949422EAE6FDE40E945B
:103480002C23EDE8F2E0ADE9B1E00E9494220E9425
:10349000D9240E949C1AA4E2B1E088278C93A4E26C
:1034A000B1E08C91803011F40C949B1AE4E2F1E0CD
:1034B000A0EAB0E00E94D924E4E2F1E001E0A4E255
:1034C000B1E00E94E524A4E2B1E0E2EFFBE40E9457
:1034D000392581E009F080E08F93A4E2B1E0EEEBC2
:1034E000FBE40E94392581E009F080E09F91892B5F
:1034F000882311F40C949B1AA0EAB0E00E943325B3
:10350000EA2FFB2F3397F0400FEFA0EAB0E00E94C4
:10351000E524A0EAB0E00E94A724AFE9B0E00C9354
:10352000E0E0F0E0AFE9B0E07BE70E94F324A4E242
:10353000B1E088278C930895E2E8FDE40E94D2224E
:1035400082E20E94DC22AAEFB2E00E94CC2282E258
:103550000E94DC220E94D92288EC90E00E9417236E
:10356000ADE9B1E00E94CC228AE10E94DC220E94F7
:10357000D9228AE10E94DC22E1E0F0E00E94E02210
:103580008DE00E94DC220E94D922DA9884E690E045
:103590000E941723DA9A82E390E00E941723A3E89F
:1035A000B2E08C918F5F8C93009183020A3011F00E
:1035B0000C94C51A80E080938302089583E0E0E3D1
:1035C0000E948D23002762FA0EF401E041E0041707
:1035D00011F00C94201B8FEF80939202A3E9B2E0CC
:1035E000ECE8FDE40E942C235A924A9280E0A42D3C
:1035F000B52D8C9381E00E9489225A924A9281E0F3
:10360000A42DB52D8C9381E00E9489220E94DC09B3
:10361000249682E00E9485225A924A92E3E9F2E0DF
:10362000A42DB52D0E94D92486E00E9489220E94F3
:103630008D0A229686E00E94852208950C94CA1B6A
:103640006CEC83E0E0E3BB27A6E121E02A930E9433
:10365000C02364E483E0E0E3BB27A6E121E02A93F2
:103660000E94C0238EEE92E00E94172383E0E0E3E5
:103670000E948D236CEC83E0E0E3BB27A6E121E010
:103680002A930E94C0236EEB83E0E0E3BB27A6E110
:1036900021E02A930E94C023BB27A6E183E0E0E358
:1036A00021E02A930E94EA23A9E9B2E05C93BB27B8
:1036B000A6E183E0E0E321E02A930E94EA23AAE95D
:1036C000B2E05C9300919A02083F18F011F00C945C
:1036D0006B1B0C94811B0FEF40919902041BA9E90D
:1036E000B2E00C930FEF40919A02041BAAE9B2E0FA
:1036F0000C93A3E9B2E0EAE7FCE40E942C230C94CB
:10370000871BA3E9B2E0E0EAFCE40E942C230091CD
:10371000990240E10E942325ABE9B2E00C930091AD
:103720009A0240E1049FACE9B2E00C9200919B0246
:1037300040919C02040FA2E9B2E00C93A3E9B2E02D
:10374000EAE7FCE40E94392511F00C94AE1B0091CD
:103750009B0241E0040FA2E9B2E00C93A3E9B2E0BE
:10376000E0EAFCE40E94392581E009F080E08F93D3
:1037700000919202003081E009F080E09F9189235E
:10378000882311F40C94CA1BA3E9B2E0E8E7FCE437
:103790000E942C2340919F0000919202041710F484
:1037A0000C94D81B92988091AA0080688093AA00FC
:1037B0000027AAEAB0E08C9187FB0EF401E041E01B
:1037C000041781E009F080E08F9340919F00009101
:1037D0009202041781E008F080E09F9189238823FA
:1037E00011F40C94F91B929A8091AA008F77809320
:1037F000AA00ADE9B2E0E2E9F2E00E945D24EDE961
:10380000F2E0ACE7B7E00E94D924ECE7F7E0ADE9DD
:10381000B2E01127222700E033270E9440230091C5
:1038200092020F3F11F00C94191CADE9B2E0882709
:103830008C935A924A9280E0A42DB52D8C9381E00E
:103840000E9489225A924A9281E0A42DB52D8C9330
:1038500081E00E9489220E94DC09249682E00E9475
:1038600085225A924A92A42DB52DE2ECFCE40E94E6
:103870002C238FE00E9489220E948D0A22968FE0DD
:103880000E9485225A924A9280E0A42DB52D8C93F5
:1038900081E00E9489225A924A9281E0A42DB52D9E
:1038A0008C9381E00E9489220E94DC09249682E0A8
:1038B0000E9485225A924A92E3E9F2E0A42DB52DA6
:1038C0000E94D92486E00E9489220E948D0A2296B5
:1038D00086E00E9485225A924A9281E0A42DB52D5D
:1038E0008C9381E00E9489225A924A9281E0A42D11
:1038F000B52D8C9381E00E9489220E94DC092496D8
:1039000082E00E9485225A924A92EDE9F2E0A42DCB
:10391000B52D0E94D92485E00E9489220E948D0A3B
:10392000229685E00E948522009192020F3F11F0BD
:103930000C94C51C5A924A9283E0A42DB52D8C9309
:1039400081E00E9489225A924A9281E0A42DB52DED
:103950008C9381E00E9489220E94DC09249682E0F7
:103960000E9485225A924A92A42DB52DE2E9FDE4E7
:103970000E942C2383E00E9489220E948D0A2296B5
:1039800083E00E9485220C94EE1C5A924A9283E0B6
:10399000A42DB52D8C9381E00E9489225A924A92DF
:1039A00081E0A42DB52D8C9381E00E9489220E9494
:1039B000DC09249682E00E9485225A924A92A42D24
:1039C000B52DE6E9FDE40E942C2383E00E948922C4
:1039D0000E948D0A229683E00E948522A6EAB0E02A
:1039E000EFE9F0E00E945D24E6EAF0E0ACE7B7E042
:1039F0000E94D924ECE7F7E0A6EAB0E011272227DD
:103A000000E033270E9440235A924A9286E0A42D78
:103A1000B52D8C9381E00E9489225A924A9281E0CE
:103A2000A42DB52D8C9381E00E9489220E94DC098F
:103A3000249682E00E9485225A924A92A42DB52DA6
:103A4000ECEAFCE40E942C2382E00E9489220E947E
:103A50008D0A229682E00E9485225A924A9288E03C
:103A6000A42DB52D8C9381E00E9489225A924A920E
:103A700081E0A42DB52D8C9381E00E9489220E94C3
:103A8000DC09249682E00E9485225A924A92A42D53
:103A9000B52DE0EAFCE40E942C2382E00E948922FA
:103AA0000E948D0A229682E00E9485225A924A92B2
:103AB00089E0A42DB52D8C9381E00E9489225A9231
:103AC0004A9281E0A42DB52D8C9381E00E94892239
:103AD0000E94DC09249682E00E9485225A924A9232
:103AE000E6EAF0E0A42DB52D0E94D92484E00E94DE
:103AF00089220E948D0A229684E00E9485225A9291
:103B00004A928BE0A42DB52D8C9381E00E948922EE
:103B10005A924A9281E0A42DB52D8C9381E00E94A7
:103B200089220E94DC09249682E00E9485225A9212
:103B30004A92A42DB52DE6E9FDE40E942C2383E0F2
:103B40000E9489220E948D0A229683E00E9485228B
:103B50000895EAE9FDE40E94D2220E94D92284EF6E
:103B600091E00E941723AEE3B2E0BA93AA930E94B9
:103B7000B515229684E690E00E941723AEE3B2E0EA
:103B8000BA93AA930E94B5152296EEE3F2E0ABEA4F
:103B9000B2E00E94D9248CE0EBEAF2E009E00A935B
:103BA000ABEAB2E00E94DE245A924A9280E0A42D51
:103BB000B52D8C9381E00E9489225A924A9280E02E
:103BC000A42DB52D8C9381E00E9489220E94DC09EE
:103BD000249682E00E9485225A924A92A42DB52D05
:103BE000E4EAFDE40E942C238CE00E9489220E94DA
:103BF0008D0A22968CE00E9485225A924A9280E099
:103C0000A42DB52D8C9381E00E9489225A924A926C
:103C100080E0A42DB52D8C9381E00E9489220E9422
:103C2000DC09249682E00E9485225A924A92EBEAAD
:103C3000F2E0A42DB52D0E94D92485E10E948922AD
:103C40000E948D0A229685E10E9485220E94F3152A
:103C500008955A924A928BE0A42DB52D8C9381E061
:103C60000E9489225A924A9280E0A42DB52D8C930D
:103C700081E00E9489220E94DC09249682E00E9451
:103C800085225A924A92A42DB52DE2EAFCE40E94C4
:103C90002C2382E00E9489220E948D0A229682E0D3
:103CA0000E948522E0EBFDE40E94D2220E94D922EC
:103CB0008CE291E00E941723AEE3B2E0BA93AA939C
:103CC0000E94B515229684E690E00E941723AEE389
:103CD000B2E0BA93AA930E94B5152296EEE3F2E001
:103CE000A3EAB2E00E94D92487E0E3EAF2E002E02E
:103CF0000A93A3EAB2E00E94DE24A3EAB2E00E94A3
:103D0000A724AAEAB2E00C935A924A928CE0A42D1E
:103D1000B52D8C9381E00E9489225A924A9280E0CC
:103D2000A42DB52D8C9381E00E9489220E94DC098C
:103D3000249682E00E9485225A924A92A42DB52DA3
:103D4000E2E9FDE40E942C2383E00E9489220E9484
:103D50008D0A229683E00E9485220091AA020030FB
:103D600080E010F009F081E08F930091AA02043006
:103D700081E008F080E09F918923882311F40C945E
:103D8000EC1E5A924A928CE0A42DB52D8C9381E0C2
:103D90000E9489225A924A9280E0A42DB52D8C93DC
:103DA00081E00E9489220E94DC09249682E00E9420
:103DB00085225A924A92A42DB52DE8EBFDE40E948B
:103DC0002C2383E00E9489220E948D0A229683E0A0
:103DD0000E9485220C94E51F0091AA02043080E025
:103DE00010F009F081E08F930091AA02093081E080
:103DF00008F080E09F918923882311F40C942B1FF5
:103E00005A924A928CE0A42DB52D8C9381E00E94A9
:103E100089225A924A9280E0A42DB52D8C9381E09C
:103E20000E9489220E94DC09249682E00E94852259
:103E30005A924A92A42DB52DECEBFDE40E942C235E
:103E400083E00E9489220E948D0A229683E00E94CC
:103E500085220C94E51F0091AA02093080E010F041
:103E600009F081E08F930091AA020F3081E008F001
:103E700080E09F918923882311F40C946A1F5A9241
:103E80004A928CE0A42DB52D8C9381E00E9489226A
:103E90005A924A9280E0A42DB52D8C9381E00E9425
:103EA00089220E94DC09249682E00E9485225A928F
:103EB0004A92A42DB52DE0ECFDE40E942C2383E072
:103EC0000E9489220E948D0A229683E00E94852208
:103ED0000C94E51F0091AA020F3080E010F009F069
:103EE00081E08F930091AA02003281E008F080E027
:103EF0009F918923882311F40C94A91F5A924A9206
:103F00008CE0A42DB52D8C9381E00E9489225A92D9
:103F10004A9280E0A42DB52D8C9381E00E948922E5
:103F20000E94DC09249682E00E9485225A924A92DD
:103F3000A42DB52DE4ECFDE40E942C2383E00E9427
:103F400089220E948D0A229683E00E9485220C9489
:103F5000E51F0091AA02003081E009F080E08F9314
:103F60000091AA02033681E009F080E09F91892B3D
:103F7000882311F40C94E51F5A924A928CE0A42DE8
:103F8000B52D8C9381E00E9489225A924A9280E05A
:103F9000A42DB52D8C9381E00E9489220E94DC091A
:103FA000249682E00E9485225A924A92A42DB52D31
:103FB000E0E9FCE40E942C2382E00E9489220E9416
:103FC0008D0A229682E00E9485220E94F3150895B0
:103FD000E8ECFDE40E94D2220E94D92280E991E01F
:103FE0000E941723AEE3B2E0BA93AA930E94B515DC
:103FF000229680E991E00E941723AEE3B2E0BA93E3
:10400000AA930E94B515229682E1EEE3F2E005E064
:104010000A93A5EDB2E00E94DE245A924A9280E013
:10402000A42DB52D8C9381E00E9489225A924A9248
:1040300085E0A42DB52D8C9381E00E9489220E94F9
:10404000DC09249682E00E9485225A924A92A42D8D
:10405000B52DE2ECFCE40E942C238FE00E94892223
:104060000E948D0A22968FE00E9485225A924A92DF
:1040700080E0A42DB52D8C9381E00E9489225A9274
:104080004A9285E0A42DB52D8C9381E00E9489226F
:104090000E94DC09249682E00E9485225A924A926C
:1040A000E5EDF2E0A42DB52D0E94D92485E10E9412
:1040B00089220E948D0A229685E10E9485220E9413
:1040C000F3150895E2EDFDE40E94D222AAEFB2E0DA
:1040D0000E94CC22EAEAFCE40E94D2220E94D92269
:1040E00084E690E00E9417230E94F3150895E6ED00
:1040F000FDE40E94D2220E94D922E1E0F0E00E9479
:10410000E022AEE3B2E0BA93AA930E94B5152296DC
:10411000AEE3B2E0BA93AA930E94B5152296AEE33D
:10412000B2E0BA93AA930E94B5152296EEE3F2E0AC
:10413000ADE9B1E00E94D9240E949C1A0E94F315B7
:1041400008950027AAEAB0E08C9186FB0EF401E006
:1041500040E0041711F00C94B520A7E8B2E0E2EDBE
:10416000FCE40E942C230C94BB20A7E8B2E0E2E11F
:10417000FDE40E942C230027A0E3B0E08C9184FB97
:104180000EF401E040E0041711F00C94C9200C94E7
:10419000DD20E2E0F0E00E94E0220027A0E3B0E0B2
:1041A0008C9184FB0EF401E041E0041711F00C94B3
:1041B000DD200C9499000C94DD200E94F3158AE018
:1041C00090E00E94172308950027A0E3B0E08C91AF
:1041D00087FB0EF401E041E0041711F00C9460211C
:1041E000D99A5A924A9280E0A42DB52D8C9381E001
:1041F0000E9489225A924A9284E0A42DB52D8C9374
:1042000081E00E9489220E94DC09249682E00E94BB
:1042100085225A924A92A42DB52DE2ECFCE40E942C
:104220002C238FE00E9489220E948D0A22968FE023
:104230000E9485225A924A9280E0A42DB52D8C933B
:1042400081E00E9489225A924A9284E0A42DB52DE1
:104250008C9381E00E9489220E94DC09249682E0EE
:104260000E9485225A924A92A42DB52DE0EEFDE4DB
:104270000E942C238FE00E9489220E948D0A2296A0
:104280008FE00E948522ABE8B2E0E6E8FBE40E9402
:104290002C23E1E0F0E00E94E02200918602003051
:1042A00011F00C945E21ADE9B1E0E0EFFDE40E9475
:1042B0002C230E949C1A81E0809386020C9490210A
:1042C0005A924A9280E0A42DB52D8C9381E00E94F1
:1042D00089225A924A9284E0A42DB52D8C9381E0D4
:1042E0000E9489220E94DC09249682E00E94852295
:1042F0005A924A92A42DB52DE8EFFDE40E942C239A
:104300008FE00E9489220E948D0A22968FE00E94EF
:104310008522ABE8B2E0E4E8FBE40E942C23D998C4
:1043200000918602003011F00C94C7215A924A92F3
:104330008DE0A42DB52D8C9381E00E9489225A92A4
:104340004A9284E0A42DB52D8C9381E00E948922AD
:104350000E94DC09249682E00E9485225A924A92A9
:10436000A42DB52DE8E7FCE40E942C2382E00E94F6
:1043700089220E948D0A229682E00E948522ADE861
:10438000B2E0E8E0FEE40E942C230C94F6215A925D
:104390004A928DE0A42DB52D8C9381E00E94892254
:1043A0005A924A9284E0A42DB52D8C9381E00E940C
:1043B00089220E94DC09249682E00E9485225A927A
:1043C0004A92A42DB52DE4E9FCE40E942C2382E05E
:1043D0000E9489220E948D0A229682E00E948522F4
:1043E000ADE8B2E0ECE0FEE40E942C230E94F3155D
:1043F0008AE090E00E9417230895E0E1FEE40E9425
:10440000D2220E94D9228AE090E00E941723AEE3D4
:10441000B2E0BA93AA930E94B51522968AE090E082
:104420000E941723AEE3B2E0BA93AA930E94B51597
:10443000229686E1EEE3F2E00CE00A93ABEAB0E00C
:104440000E94DE24EEE3F2E0A4E2B1E00E94D9246F
:10445000E4E2F1E004E0A4E2B1E00E94E524A4E299
:10446000B1E0EAE1FEE40E94392511F00C947822D3
:104470008AE090E00E941723AEE3B2E0BA93AA93D9
:104480000E94B5152296EEE3F2E0A4E2B1E00E94AC
:10449000D924E4E2F1E00EE0A4E2B1E00E94E524D8
:1044A000DA9884E690E00E941723DA9A82E390E09B
:1044B0000E941723A3E8B2E08C918F5F8C93009148
:1044C00083020A3011F00C94502280E08093830222
:1044D000E4E4FBE40E94D22282E20E94DC22EEE4C9
:1044E000FBE40E94D22282E20E94DC220E94D922B6
:1044F00084E690E00E9417230E94F31508958E2E03
:104500009F2E0895E82DF92D0895481A8827580AF6
:104510000895480E8827581E0895ED91FC91EF5F8D
:10452000FF4FFC93EE9308958F938D918823E9F7C5
:1045300011978F91089580919E00882309F081E062
:10454000089580919E00882309F408950F929F9307
:10455000AF93BF937F9380919E008823E1F3F894FB
:1045600080919E008A9580939E0090919C00A0E689
:10457000B0E0A90F0024B01D8C9193959C3309F4F1
:10458000992790939C0078947F91BF91AF919F91D0
:104590000F900895ACE7B7E08D91882311F00CD00F
:1045A000FBCF08950E943223802D11F005D0FACF61
:1045B00008958DE001D08AE05D9BFECF8CB908950F
:1045C00088EE93E034D03197D9F708953197F1F719
:1045D00008950E94F9228D910E94FD229A95D9F7A3
:1045E0000E94FC220895DB98D39ADC98D49AD19843
:1045F0000895DB98DC980895089508E0880F10F47A
:10460000DC9A02C0DC980000DB9A0058005EF0F3F0
:10461000DB980058005EF0F3C99983950A9571F70D
:104620000895689462F80895E89462F80895EF9305
:10463000FF93EE27E82BE92B31F0E0EAFFE031971A
:10464000F1F70197D1F7FF91EF9108955A924A92AD
:10465000480E8827581E08950E9432230D9200208C
:10466000D9F70895C89531960020089591E08823E0
:1046700021F08894991F8A95E9F7892F90950895DC
:104680002E2E3F2E992781918D3209F09395882304
:10469000D1F79A95E22DF32D112361F0091718F047
:1046A00011F0101B01C0191B28F021F080E28D933E
:1046B0001A95E9F780818D3219F48D93319604C0F3
:1046C000222311F08BE28D93091738F031F0091B8A
:1046D00021F080E38D930A95E9F781918D938823EA
:1046E000E1F7332351F0EA2FFB2F319633958E916A
:1046F00082933A95E1F78EE28C9308950181082B1D
:104700000183128119231283EF93FF93E4E0F0E019
:104710000E94E622FF91EF9108950E941123FF2746
:104720000E943623EBDFEF93FF93ECE7F7E00E9464
:10473000E622FF91EF91182B128309230183EF9357
:10474000FF93E4E6F1E00E94E622FF91EF911081F1
:10475000182369F4EF93FF93ECE7F7E00E94E62259
:10476000FF91EF911081182311F00E941423EF9311
:10477000FF93ECE7F7E00E94E622FF91EF910895A6
:104780000E943623FF2729915D9148E0B7DFEF9320
:10479000FF93E4E0F0E00E94E622FF91EF9157954D
:1047A00010F4182B1283EF93FF93ECEEF0E00E94CD
:1047B000E622FF91EF91182B1283EF93FF93E4E031
:1047C000F0E00E94E622FF91EF914A95F9F62A95D2
:1047D000D9F608950E943623FF27299148E05527EE
:1047E0008DDF09230183EF93FF93E4E1F0E00E9462
:1047F000E622FF91EF9188941081182309F0089424
:104800005795EF93FF93E0EBF0E00E94E622FF91D3
:10481000EF914A9529F75D932A9501F708957F93C3
:104820000F93AF93BF938F939F938FB78F93809185
:104830009E000CE3081B21F49CB10E94112312C0BE
:1048400000919D00A0E6B0E077279CB1A00FB71FB4
:104850009C93839580939E0003950C3309F4002765
:1048600000939D008F918FBF9F918F91BF91AF91CA
:104870000F917F911895040F151F261F371F08955C
:10488000000F111F221F331F0895009510952095CA
:1048900030950F5F1F4F2F4F3F4F089501911081AB
:1048A0000EC001911191219130810BC001911081B5
:1048B00017FF05C03FEF2FEF04C00081112722270B
:1048C000332737FF03C0E1DF8DE28D93CF93DF9372
:1048D000CF92DF92EF92AA24BB24CC24DD24EE24D5
:1048E00040E2CAE0DD2755E093E38881890F87FD28
:1048F0009F7083FD907F891B89935A95A9F7C0DF2C
:10490000AA1CBB1CCC1CDD1CEE1C4A9551F7E8947C
:10491000EFE0FF2782910ED0EB30E0F71EF06894B5
:104920008A2D0CD088278D93EF90DF90CF90DF9168
:10493000CF910895982F829501D0892F8F70805D37
:1049400026F0803309F4089568948D930895002724
:104950001127222733271DD08A3328F4803318F0FB
:1049600005D015D0F9CF0EF490CF089580538F93D2
:10497000402F512F622F732F83DF82DF7CDF80DF98
:104980008F919927080F191F291F391F08958D919D
:104990000895E894FCDF8032E9F38B32D9F3893053
:1049A000C9F38D3211F46894F2CF089588278D935E
:1049B000089581918D938823E1F70895099191914C
:1049C000992351F08A95D9F7319781918D930A9562
:1049D00019F08823D1F70895E9CFE199FECFEEBB16
:1049E000FFBB3196089591E001C092E07B3751F40E
:1049F0007FB7F894F2DF8D918DBBE29AE19A9A9598
:104A0000C9F77FBF77270895E8DF8D917B3729F4B9
:104A10008DBBE29AE19A8823B9F77727089591E050
:104A200001C092E0DADFE09A8DB38D939A95D1F7C9
:104A30000895D3DFE09A8DB38D93882319F09A956A
:104A4000C1F79D930895FF93881BF9E0001FFA9525
:104A500011F4FF910895881F841B18F4840F889423
:104A6000F5CF0894F3CF8FEF83959D919923E1F7CC
:104A70000895689401C0E894AF93BF938D9116F0A8
:104A8000919103C00E943223902D891718F011F4E0
:104A90008823A1F7BF91AF9108955265762E3133E7
:104AA000303132332E64000047534D2053494D3985
:104AB000303044002D2D2D2D2D2D2D2D2D2D2D2D36
:104AC0002D2D000041565270726F6A6563742E720C
:104AD0007500C2EAEBFEF7E5EDE8E5202020202096
:104AE0000000DAFAFAFAFAFAFAFAFAFAFAFAFADB59
:104AF0000000D900D800D600D700D0E5E3E8F1F2F5
:104B0000F0E0F6E8FF2020200000DA00CEF7E8F120
:104B1000F2EAE020E1F3F4E5F0E0000041540000A7
:104B2000C2E5F0E8F4E8EAE0F6E8FF2041540000CE
:104B30004F4B0000D3E4E0EBE5EDE8E520534D53A7
:104B40002020000041542B434D4744413D00444543
:104B50004C20414C4C00C90053494D393030442061
:104B6000E3EEF2EEE221000041542B434D47463D77
:104B7000310041542B434C49503D31004154533096
:104B80003D32000030003100320033003400350087
:104B9000360037003800390041004200430044002D
:104BA000450046004700480049004A004B004C00C1
:104BB0004D004E004F005000510052005300540071
:104BC000550056005700580059005A006100620015
:104BD00063006400650066006700680069006A00A1
:104BE0006B006C006D006E006F0070007100720051
:104BF00073007400750076007700780079007A0001
:104C0000C000E000C100E100C200E200C300E30018
:104C1000C400E400C500E500A800B800C600E60036
:104C2000C700E700C800E800E900CA00EA00CB00BE
:104C3000EB00CC00EC00CD00ED00CE00EE00CF008C
:104C4000EF00D000F000D100F100D200F200D3005C
:104C5000F300D500F500F700F600D400F400F800EA
:104C6000F900DC00FC00FA00DB00FB00DD00FD00C9
:104C7000DE00FE00DF00FF0020002D002E003A00C5
:104C80003E00B0004000260027003C002A002C0017
:104C900024003D002100BD00230028005B0025000A
:104CA0002B005E003F005D0029003B002F005C00F0
:104CB0005F002B434D54000041542B434D47523D60
:104CC0000000202020202020202020202020202024
:104CD00000004F666600CAEEF2E5EB20C2DBCACBED
:104CE000202020200000CDE0F1EEF120C2DBCACB75
:104CF000202020200000CDE0F1EEF120C2CACB2020
:104D0000202020200000CAEEF2E5EB20C2DBCACB57
:104D100000004F4E0000CAEEF2E5EB20C2CACB20E5
:104D2000202020200000415453303D3000004669CF
:104D30007273746E756D626572004E756D62657228
:104D40003A200000204F4B0053494D393030440089
:104D500054656D703A00506F726F67004C6F6164FC
:104D60003A0053656E736F723A0053656E64205358
:104D70004D532066726F6D2073656E736F72733A58
:104D8000000041542B434D47533D00006572726F44
:104D9000720020200000B043000041542B434F50CC
:104DA000533F000020202020202020202020200011
:104DB00041542B43535100003E2000003C20000092
:104DC0003C4000003C26000041542B43434C4B3FE9
:104DD000000041544400415444233130302300004A
:104DE000C2F5EEE43A2031202020202020200000CF
:104DF000416C61726D210000C2F5EEE43A20302072
:104E00002020202020200000596573004E6F0000F4
:104E100041542B434D47523D31002B434D47000039
:00000001FF
